:100000000C9488000C94BF1C0C94981C0C94A500B4
:100010000C94A5000C94A5000C94A5000C94A500CC
:100020000C94A5000C94A5000C94A5000C94A500BC
:100030000C94A5000C94A5000C94A5000C94A500AC
:100040000C944E1C0C94A5000C94A5000C94A500D7
:100050000C94A5000C94A5000C94A5000C94A5008C
:100060000C94A5000C94A5000C0D0E0F10110001AE
:1000700002030405060708090A0B0100010001003C
:100080000100010001000100010001000100010068
:1000900001000100010001000100010001003050D9
:1000A00000000001010101010110101010103010BA
:1000B000101010100100000000240027002A00008A
:1000C0000000080002010000030407000000000017
:1000D00000000000000000230026002900010204A7
:1000E00008102040800102040810200102040810BA
:1000F0002000000000250028002B00040404040454
:1001000004040402020202020203030303030300C5
:1001100011241FBECFEFD8E0DEBFCDBF11E0A0E0BD
:10012000B1E0EAE4F9E402C005900D92A83CB10701
:10013000D9F722E0A8ECB1E001C01D92AA32B207C3
:10014000E1F70E94721D0C94A3240C9400008230ED
:10015000F8F4E82FF0E0EE0FFF1FE050FF4F24ED22
:1001600031E031832083813041F0809169008C7FC0
:10017000682B60936900E89A089580916900837FF5
:10018000660F771F660F771F682B60936900E99AE7
:100190000895089590E0FC01E154FF4F2491FC0183
:1001A000E352FF4F3491FC01E550FF4FE491EE2301
:1001B000C9F0222339F0233001F1A8F4213019F1DC
:1001C000223029F1F0E0EE0FFF1FEF50FF4FA59115
:1001D000B4918FB7F894EC91611126C030953E230D
:1001E0003C938FBF08952730A9F02830C9F0243000
:1001F00049F7809180008F7D03C0809180008F77C8
:1002000080938000DFCF84B58F7784BDDBCF84B54A
:100210008F7DFBCF8091B0008F778093B000D2CFDD
:100220008091B0008F7DF9CF3E2BDACFCF93DF9353
:1002300090E0FC01E352FF4F249185509F4FFC0159
:1002400084918823C9F090E0880F991FFC01EB543A
:10025000FF4FA591B491FC01EF50FF4FC591D49190
:1002600061110DC09FB7F8948C91209582238C93D7
:100270008881282328839FBFDF91CF910895623022
:1002800051F49FB7F8943C91822F809583238C93EF
:10029000E8812E2BEFCF8FB7F894EC912E2B2C9377
:1002A0008FBFEACF1F93CF93DF93182FEB0161E04D
:1002B0000E941601209739F460E0812FDF91CF91E1
:1002C0001F910C94CA00CF3FD10511F461E0F5CF26
:1002D000E12FF0E0E154FF4FE491E33031F140F4DD
:1002E000E130B1F0E230E1F0C038D1057CF7E4CF85
:1002F000E73029F1E83059F1E430B1F7809180001E
:10030000806280938000D0938B00C0938A0004C0E9
:1003100084B5806884BDC7BDDF91CF911F910895DA
:1003200084B5806284BDC8BDF7CF809180008068AD
:1003300080938000D0938900C0938800EDCF809196
:10034000B00080688093B000C093B300E5CF809187
:10035000B00080628093B000C093B400DDCF3FB79F
:10036000F8948091D2019091D301A091D401B091E1
:10037000D50126B5A89B05C02F3F19F00196A11DF8
:10038000B11D3FBFBA2FA92F982F8827BC01CD01DF
:10039000620F711D811D911D42E0660F771F881F3E
:1003A000991F4A95D1F70895FF920F931F93CF930A
:1003B000DF930E94AF012091CB013091CC01EB0182
:1003C000C21BD30B2091D8013091D901C217D3079A
:1003D00008F45FC04091DC015091DD0141305105CE
:1003E00061F0E0910502F091060220813091070250
:1003F00023233091D60123134CC07093CC0160931A
:10040000CB010091DA011091DB014230510509F472
:1004100013C14330510509F44EC14130510561F417
:100420008091CA01813009F447C0C8F1833009F4D2
:1004300082C0843009F4C9C08091DC019091DD0153
:10044000019739F1C017D10708F06DC18091C8013B
:100450008F5F8093C8018B30E0F081E090E0909353
:10046000DD018093DC0161E070E0809103020E9475
:10047000A7001092D6011092CA0182E590E09093F5
:10048000DB018093DA0183E290E09093D9018093BD
:10049000D801DF91CF911F910F91FF900895C01760
:1004A000D10730F481E08093CA01C093C901C4CF61
:1004B00084E08093CA01C0CFC017D107D0F5109255
:1004C000CA018091C8018F5F8093C8012091C90142
:1004D0008C2F0C2E000C990B821B910927FD9395F4
:1004E00097FF03C0919581959109499794F21092D5
:1004F000DD011092DC0182E990E09093DB018093B2
:10050000DA0182E590E09093D9018093D8011092AE
:10051000C801F090D7016F2D70E0809103020E9416
:10052000A7008091070293E0F91227C08093D601BB
:1005300083CF83E0BECFC017D10708F51092DD014D
:100540001092DC0182E990E09093DB018093DA0164
:1005500082E590E09093D9018093D8011092C80170
:10056000F090D7016F2D70E0809103020E94A700E8
:100570008091070233E0F316C9F280E0D7CF909163
:10058000D701933009F482E08093D70182E090E0B4
:100590009093DD018093DC0182E990E09093DB0190
:1005A0008093DA0182E590E09093D9018093D8019D
:1005B0001092E2018091C8018093E3011092DF0163
:1005C0001092E1011092E001CBCFC017D107A8F43F
:1005D0001092DD011092DC0182E990E09093DB0142
:1005E0008093DA0182E590E09093D9018093D8015D
:1005F0001092C8011092DF018CCF82E090E09093BE
:10060000DD018093DC0182E990E09093DB0180932F
:10061000DA0182E590E09093D9018093D80110929D
:10062000E2018091C8018093E3011092DF011092F2
:10063000E1011092E0016DCF9091DF019F5F9093F7
:10064000DF018091E001880FC017D107E0F08093AF
:10065000E001983009F0F6CEE091E201E630A9F42D
:100660001092DD011092DC0182E990E09093DB01B1
:100670008093DA0182E590E09093D9018093D801CC
:100680001092DF01D9CE8160E2CF83E090E09093B9
:10069000DD018093DC0181E08E0F8093E201909177
:1006A000E001F0E0E452FE4F90878091E10189275C
:1006B0008093E101C1CEC017D10728F51092DD016A
:1006C0001092DC011092DF0182E990E09093DB014F
:1006D0008093DA0182E590E09093D9018093D8016C
:1006E0008091E1018111B2CE88E0E2EEF1E0AAEE64
:1006F000B1E001900D928A95E1F781E08093DE01EF
:100700001092C80199CE8091E201863009F4A8CFF9
:1007100082E090E09093DD018093DC011092DF0194
:100720001092E00189CE1092C801B3CE2FB7F89491
:100730006091CE017091CF018091D0019091D10153
:100740002FBF089508950895CF93DF93FC012BEAFE
:10075000629F212D1124269532E1239FC00111248F
:10076000A481B581A80FB91F322F330F230F621B4D
:10077000462F50E0ED0125E0629FC00DD11D1124F0
:100780002B8123FF1EC011962C9111973FEF320F42
:1007900011963C93222319F0208521502087A481B3
:1007A000B581A80FB91F65E0649F9001659F300D6A
:1007B0001124A20FB31F13962C911397277F139622
:1007C0002C93A481B581A80FB91F25E0249FE001D7
:1007D000259FD00D1124CA0FDB1F2B8124FF1EC0C3
:1007E00012962C9112973FEF320F12963C932223D0
:1007F00019F0218521502187A481B581A80FB91F47
:1008000065E0649F9001659F300D1124A20FB31F16
:1008100013962C9113972F7E13962C93A481B58158
:10082000A80FB91F65E0649F9001659F300D1124EA
:10083000A20FB31F13964C9113974E7F13964C93B0
:10084000A481B581A80FB91FA20FB31F13964C91B5
:1008500013974D7F13964C93A481B581A80FB91FB0
:10086000A20FB31F13964C9113974B7F13964C9383
:10087000A481B581A80FB91FA20FB31F16961C92B1
:1008800044815581480F591F240F351FD9011796F0
:100890001C920480F581E02DE80FF91F80818160B2
:1008A0008083DF91CF9108952F923F924F925F9274
:1008B0006F927F928F929F92AF92BF92CF92DF9270
:1008C000EF92FF920F931F93CF93DF93CDB7DEB7D5
:1008D0002B970FB6F894DEBF0FBECDBF9B878A87DC
:1008E000DC0112968C918F3F09F412C180E0F2E195
:1008F0002F2EA3E03A2EEA85FB859381891708F015
:1009000082C0282F30E0829D80011124E480F58090
:10091000E00EF11ED7019C9190FF5EC0A681B781C9
:1009200012964D915C9113972417350708F054C027
:10093000F7019781448550E070E060E0762F652FE5
:10094000542F4427692B9189492B4B01AA24BB249E
:10095000452E562E672E7724E42CF42E18969C9163
:100960001897992391F0C92ED12CC89C7001C99C6D
:10097000F00CD89CF00C11248F2C949D2001112494
:10098000E52C949FA0011124F52E1E964C911E97E4
:1009900019966D917C911A971B969C911B97491300
:1009A00026C09B01839D200D311D11241B964C9167
:1009B0001B97420F532F511DFA0180821C964C91B8
:1009C0001C97420F532F511DFA01E0821D969C91F6
:1009D000290F311DD901FC92EA85FB85A481B581DF
:1009E000A00FB11F9C919E7F9C938F5F84CF220F9D
:1009F000331F220F331F260F371F420F532F511D56
:100A0000FA011082D3CFEA85FB8506811781D801D0
:100A100019968D919C91892B09F47AC0F801C784AD
:100A2000D088E188F2880E94AF016C157D058E05A3
:100A30009F0548F40E94AF01D8011F966D937D93E6
:100A40008D939C9352970E94AF01F801C784D08880
:100A5000E188F2886C197D098E099F096C3271401A
:100A600081059105D8F2F894D80114968D919C9146
:100A700015979A8389831996ED91FC917F01BFEFB9
:100A8000EB1AFB0A80818987F80190810388F48939
:100A9000E02DD80155968C91992309F452C090818C
:100AA000982B98879081809589238F838F818C8361
:100AB00088E08B8358856F8149853B812C818981B2
:100AC0009A81D701508347FD252F3A952083262F01
:100AD00039F0441F00C000006083000000C0F2CF66
:100AE00038E04D9160830000019761F7D80154967A
:100AF000FC93EE93539749873B832C839A83898396
:100B000078940E94AF01F8016787708B818B928B7C
:100B10002B960FB6F894DEBF0FBECDBFDF91CF91FD
:100B20001F910F91FF90EF90DF90CF90BF90AF900B
:100B30009F908F907F906F905F904F903F902F90FD
:100B400008959081982B98879081809589238F8331
:100B50008F818E8388E08D8358856F8149853D81A3
:100B60002E8189819A81D701508347FD252F00C0AE
:100B700000C0208300C000C000C000C000C060836F
:100B80000000262F3A9541F0441F000000C000C02D
:100B900000C000C000C0E8CF38E04D9100C06083C5
:100BA00000C0019709F7D8015496FC93EE93539730
:100BB00049873D832E83A2CFDC012BEA629F212D42
:100BC00011242695822F880F820F681B4031A9F0CF
:100BD000403319F1413081F41496ED91FC9182E19A
:100BE000289FE00DF11D112485E0689FE00DF11DA7
:100BF000112483818160838308951496ED91FC9183
:100C000082E1289FE00DF11D112485E0689FE00D31
:100C1000F11D112483818260EECF82E1289F900133
:100C200011241496ED91FC911597E20FF31F85E0C6
:100C3000689FB0011124E60FF71F838182608383D0
:100C40001496ED91FC91E20FF31FE60FF71F8381DD
:100C50008460D1CFDF92EF92FF920F931F93CF93D7
:100C6000DF93EC018E81882309F449C0F12C96E0D2
:100C7000E92E0FEF10E08A81F81608F040C0FE9CC4
:100C8000C0011124EB81FC81E80FF91F208120FFB6
:100C900028C021FF26C023812F5F2383EB81FC81A5
:100CA000273008F5E80FF91FA381B0E0A05BBE4F25
:100CB0002C913281239F202D11242583EB81FC81EF
:100CC000E80FF91F658128E0629FB001112481813E
:100CD0009D8190FF04C09801261B370BB9010E942B
:100CE0005201F394C8CF2E81222311F021502E837C
:100CF000E80FF91F20812D7F20832481DECF8F8193
:100D0000882309F44DC0F12C86E0E82E0FEF10E0A7
:100D1000DD24DA948A81F81608F042C0FE9CC001F6
:100D20001124EB81FC81E80FF91F208120FF28C0EE
:100D300022FF26C0238121502383EB81FC812223C3
:100D400009F1E80FF91FA381B0E0A05BBE4F2C9121
:100D50003281239F202D11242583EB81FC81E80F14
:100D6000F91F658138E0639FB001112481819D8165
:100D700090FF04C09801261B370BB9010E94520155
:100D8000F394C8CF2F81211108C0DF82E80FF91F2B
:100D900020812B7F20832481DFCF22502F83F6CF29
:100DA000DF91CF911F910F91FF90EF90DF90089509
:100DB000DC0112967C91129730E020E090E07917E8
:100DC000E1F11396ED91FC911497E20FF31F8181ED
:100DD000A9014A5F5F4F86132DC0908190FF25C007
:100DE00091FF0AC016969C911697915016969C9367
:100DF000169790819D7F9083908192FF0AC01796ED
:100E00009C911797915017969C93179790819B7F71
:100E1000908390819E7F9083148213964D915C9174
:100E20001497240F351FF901158215966C91617086
:100E30000C94CA009F5F9A01C2CF0895CF93DF93AD
:100E4000FC01862F5281D0E0C0E090E0591791F16B
:100E5000A381B481AC0FBD1F11963C911197BE01C7
:100E60006A5F7F4F381365C09C9190FF42C0442356
:100E700031F18FEF820F8F3100F5822F880F880FAD
:100E8000880F14968C93A381B481AC0FBD1F8C91F5
:100E900081FD03C086818F5F86838C9182608C93F5
:100EA000211101C020E212962C9383819481C80FF6
:100EB000D91F1B82DF91CF9108958FEFE2CF91FF71
:100EC00006C08681815086838C918D7F8C938C9116
:100ED00082FD03C087818F5F87838C9184608C93B0
:100EE00014961C9283819481C80FD91F87E08B834D
:100EF000E1CF6581962F91705FEF520F5F3190F4D3
:100F0000442381F038E0239FB0011124992331F06C
:100F10002FEF30E0A901461B570BBA01DF91CF91AB
:100F20000C945201642F6927832FDF91CF910C9489
:100F3000CA009F5FEB018ACF0F931F93CF938C0161
:100F4000C62FDC0112969C9130E020E080E09817DB
:100F500061F0D8011396ED91FC91E20FF31F2A5F27
:100F60003F4F41814F3F71F4C18361E08C2F0E945C
:100F70001601F801658161708C2FCF911F910F913F
:100F80000C94CA008F5FE3CFDC0112968C9112970C
:100F900030E020E090E0891799F01396ED91FC91F4
:100FA0001497E20FF31F2A5F3F4F5181561306C07B
:100FB000413031F480818160808308959F5FEBCF61
:100FC000089508950895DC0113964C91139750E00D
:100FD00030E020E0241735079CF4C901880F991FE1
:100FE0001496ED91FC911597E80FF91F0190F0818F
:100FF000E02D9681947F9B7F96832F5F3F4FEACFB2
:1010000008952F923F924F925F926F927F928F92AC
:101010009F92AF92BF92CF92DF92EF92FF920F9387
:101020001F93CF93DF9300D000D0CDB7DEB7213030
:10103000310509F03FC0DC011496CC90B0E0A0E08F
:10104000F3E0BF2EAA24A394AC15A0F5FC01828086
:1010500093808A0E9B1EF4011081FB01868097808D
:101060001B9D800C911C1124F401128112FBDD24C4
:10107000D0F8DA24D016A1F080809180F401D680D7
:10108000D1FA662460F8011103C0D0FA662460F832
:10109000712C672829F04130510521F410FF07C059
:1010A0001196D2CF41155105D9F711FDF9CF30E096
:1010B00020E0F6CFDC0115962C904090180250905D
:1010C0001902C0900E02D0900F021C821B82EDE02C
:1010D0003E2EBB81B21508F08BC0DC01ED91FC9176
:1010E000AB81BC81EA0FFB1F1081DB011896ED91EB
:1010F000FC91139DE00DF11D11241485211531057E
:10110000A1F0A081B181109781F010FF0EC016965A
:10111000AC91A1FBEE24E0F8011103C0A0FBEE248A
:10112000E0F8F12CEF2809F45DC012FBAA27A0F922
:10113000B1E0AB27A01709F455C0728441305105C6
:1011400011F411FD4DC0172D7384A12FB0E0AA0F2B
:10115000BB1FAE0FBF1F171508F044C01296EC91CD
:101160001297EF3FD1F1F0E04F01880C991CF2018A
:10117000A384B484F401EA0DFB1DA080B180139612
:101180009C901397E0E26E2E992071F0F60180801A
:10119000612C891448F09A94998281809280F4019C
:1011A0006980E60DF11D6080992493942115310525
:1011B00009F4912CF501F181FA83F2FB882480F87F
:1011C00098288F2E90FA82F8F50181822115310539
:1011D00021F09380961408F463821F5F1296BBCFB0
:1011E00010E0B3CFAB81BC811196BC83AB8371CFD0
:1011F0000F900F900F900F90DF91CF911F910F9153
:10120000FF90EF90DF90CF90BF90AF909F908F9026
:101210007F906F905F904F903F902F9008958F92A6
:101220009F92AF92BF92CF92DF92EF92FF920F9375
:101230001F93CF93DF93E0901C02F0901D02E0918A
:101240001A02F0911B0280809180D0E0C0E0D701AB
:1012500013968C9113978C171D0639F134F114965F
:10126000ED91FC91CE01880F991FE80FF91FA08026
:10127000B180F501268122FF08C0217000E030E036
:10128000A401B701C5010E940108D50116962C9151
:1012900023FF09C02695217001E030E0A401B701C9
:1012A000C5010E9401082196D2CF00911802109129
:1012B0001902F12CE12CF8018285F816E8F58F2D42
:1012C00090E0880F991F0384F485E02DE80FF91F43
:1012D000C081D181898182FB442740F92B81869589
:1012E0008170481303C08A81821721F1898140FBF4
:1012F00081F989832A83E0911802F091190280FB19
:10130000CC24C0F8D12CC601880F991FE80FF91F13
:1013100081819281DC01ED91FC910480F581E02DC9
:101320006881099581E099819B7F99831B82E82AD6
:10133000F394C1CF80E0F7CFEE20B1F0C0E0F80128
:101340008081C81788F4EC2FF0E0EE0FFF1FE00F4C
:10135000F11F81819281DC01ED91FC910680F78182
:10136000E02D0995CF5FEBCFDF91CF911F910F91CA
:10137000FF90EF90DF90CF90BF90AF909F908F90B5
:101380000895CF93C82F80E090E0892B51F0809191
:10139000F4018C1731F081E0C11101C080E00E949E
:1013A0000000C093F40160E070E0CB01C1110E9425
:1013B00096036093F5017093F6018093F701909383
:1013C000F80180E090E0892B59F08091F4018C17AE
:1013D00039F081E0C11101C080E0CF910C94000090
:1013E000CF910895642FA0910C02B0910D0241E0BD
:1013F00050E02130310511F050E040E0ED91FC91DA
:1014000011970084F185E02D262FBC01CD010994B0
:10141000A0910C02B0910D02ED91FC911197068004
:10142000F781E02DBC01CD010994462FA0910C025B
:10143000B0910D02ED91FC9111970480F581E02DA2
:10144000BC01CD0109940895A0910C02B0910D0248
:10145000ED91FC9111970280F381E02DBC01CD014B
:101460000994A0910C02B0910D0241E0611101C0FC
:1014700040E0ED91FC9111970190F081E02DBC01CD
:10148000CD0109940C94310A80E090E0892B29F079
:1014900080910B0283FD0C9400000895CF93DF939D
:1014A000EC0161E08B810E94CA0081E089870E9483
:1014B00096036A5F7F4F8F4F9F4F6D837E838F832D
:1014C000988783E08C83DF91CF91089580910C02FF
:1014D00090910D020C944E0A0C94660ACF92DF9202
:1014E000EF92FF92CF93DF93EC01888180FF14C0CD
:1014F000C980DA80EB80FC800E949603C61AD70A66
:10150000E80AF90A9EEF1C141D041E041F040CF4C3
:101510009FEF88818923888388818170DF91CF91B3
:10152000FF90EF90DF90CF9008950F93CB01642F41
:10153000422F202FDC01ED91FC910280F381E02D00
:101540000F910994CB01642FDC01ED91FC91019086
:10155000F081E02D422F0994CF93DF93FC01EA0143
:101560008089861799F0608B8FEF9FEF928B818B2C
:10157000138A662359F0683208F052C0613069F46A
:1015800081E1838B81E090E0928B818B83898883DA
:1015900081899289DF91CF910895613121F4638B24
:1015A00081E190E0F1CF623129F481E1838B82E126
:1015B00090E0EACF673039F486E1838B87E090E0F2
:1015C000222311F3E3CF683039F487E1838B88E07D
:1015D00090E02223C9F2DACF6D3129F489E1838BBF
:1015E0008DE190E0D1CF6E3129F489E1838B8EE1DA
:1015F00090E0CACF6F3129F489E1838B8FE190E0CD
:10160000C3CF603229F489E1838B80E290E0BCCFC4
:10161000613209F0BBCF89E1838B81E290E0B4CFE6
:1016200028ED260F283408F580E2838B822F66E0B0
:101630000E942B23382F822F90E066E070E00E94FA
:1016400037232085321708F0A1CF23E2009729F035
:1016500024E28130910509F025E2238B26E0329FB8
:10166000800D911D112488968FCF80E9860F8530DB
:1016700060F490E4938B9285891708F087CF97E404
:10168000938B90E080599F4F7FCF65578485681773
:1016900008F07CCF89E5838B70E06B587F4F728BAD
:1016A000618B74CF089508950895CF93DC0150960F
:1016B000ED91FC913097D9F0E617F707F1F4C22FBE
:1016C000E0911A02F0911B02808191818427952775
:1016D000019721F4518340830E940F09E0911A027F
:1016E000F0911B028481C81741F0C48306C0FC013D
:1016F000868597858617970711F3CF910895CF9226
:10170000DF92EF92FF920F931F93CF93DF934130BD
:10171000510519F4220F25FD2160DC011E96ED9183
:10172000FC911F97E617F70791F050968D919C91C9
:10173000009721F011E08617970751F0DF91CF91C4
:101740001F910F91FF90EF90DF90CF90089510E0E0
:101750008FEF840F853090F75527FA01E65BFE4F37
:10176000DF0111974C91F080C0911C02D0911D02B5
:10177000B0E0A0E050E030E04F1508F042C0C901F1
:101780000A2E02C0959587950A94E2F7982F9170DA
:101790006C85862F817060FD812FEB8070E060E0AA
:1017A0006E1528F080E0582B4F5F1196E5CF6B0146
:1017B000CC0CDD1CEC81FD81EC0DFD1D0190F08158
:1017C000E02D07816F5F7F4F041750F34013EACF7E
:1017D00081110CC0868184608683682F617090FBC4
:1017E00080F96917F9F2868381E0DDCF8681886010
:1017F000868381FB662760F96917A1F290FB81F966
:10180000F2CF552309F49ACFDF91CF911F910F9119
:10181000FF90EF90DF90CF900C940F090F931F93E0
:10182000CF93DF931F92CDB7DEB7009110021091D6
:101830001102D801ED91FC910190F081E02D20E0A2
:10184000AE014F5F5F4FC80109958F3F980781F048
:10185000D801ED91FC910680F781E02D4981BC0112
:10186000C80109950F90DF91CF911F910F910895B5
:1018700080E0F8CFCF93DF931F92CDB7DEB7242F50
:101880008091100290911102DC01ED91FC91019088
:10189000F081E02DAE014F5F5F4F099521E0019689
:1018A00009F420E0822F0F90DF91CF910895E42F6B
:1018B000F0E0ED55FF4F84910895E42FF0E0E256FB
:1018C000FF4F84910895D90186E04C3008F034C070
:1018D000E42FF0E0E259F34F0C945F237A0C810C73
:1018E000840C870C9C0C9C0C8A0C8D0C900C930C1B
:1018F000960C990CEEE0F1E001900D928A95E1F7DB
:101900000895E4E1F1E0F8CFEAE1F1E0F5CFE0E2BB
:10191000F1E0F2CFE6E2F1E0EFCFECE2F1E0ECCF84
:10192000E2E3F1E0E9CFE8E3F1E0E6CFEEE3F1E076
:10193000E3CFE4E4F1E0E0CFFD0111928A95E9F70D
:10194000089586ED96E0089587ED96E00895E62FD8
:10195000F0E0EE0FFF1FE658FF4F849190E00895EE
:10196000E62FF0E0E859FF4F8491089582E1089551
:101970007F928F929F92AF92BF92CF92DF92EF921F
:10198000FF920F931F93CF93DF93DC0113961C916B
:1019900013971496ED90FC90159790E080E0782EC8
:1019A0005C01AA0CBB1CAE0CBF1CE501E881F981EF
:1019B000811720F401962781261788F3309719F0B4
:1019C00087818617E9F112968C9112978117C0F1E1
:1019D000062F6D01E12FF0E0EE0FFF1FEE0EFF1E50
:1019E000F701C081D1812097B1F488E090E00E9496
:1019F0006523EC01F60180801C821D828FEF8F83AE
:101A0000912CC4010E9465239B838A83C4010E9498
:101A10006523998388830F838E81847F8B7F8E8358
:101A200081E0810FF6018383F701711630F4929102
:101A30008291938382831150F8CFF501D183C083C3
:101A4000872DDF91CF911F910F91FF90EF90DF9045
:101A5000CF90BF90AF909F908F907F9008950E94FD
:101A6000C109E2EFF1E081E087831086EBEFF1E05E
:101A700088E0DF011D928A95E9F708952F923F9241
:101A80004F925F926F927F928F929F92AF92BF928E
:101A9000CF92DF92EF92FF920F931F93CF93DF933A
:101AA00000D000D0CDB7DEB79C838B83DC011896C5
:101AB0008C91B12C882309F45EC1E12C35E0F32E22
:101AC00042E3442E512C612C712C54E1352EEB81D4
:101AD000FC818381E81608F04EC1F2E1EF9E80019F
:101AE0001124AB81BC811496ED91FC91E00FF11FA4
:101AF0008181882309F44EC090E080E0EB81FC8175
:101B000024813581200F311FF89ED001F99EB00D40
:101B10001124F901EA0FFB1F7381AC014F5F5F4F86
:101B20006A0170FF63C073FB662760F973FF5EC0D4
:101B300025812F5F2583EB81FC8144815581FA014A
:101B4000E00FF11F273040F5AE0FBF1FFC9CC00116
:101B5000FD9C900D1124E80FF91FE081F0E0E05B9F
:101B6000FE4F808114969C911497899F802D11249B
:101B700017968C93AB81BC811496ED91FC91E00F8C
:101B8000F11F808181608083B62EC601833091056C
:101B900009F0B4CFE3949BCF21813FEF320F318323
:101BA000222341F0AB81BC8118962C9118972150CB
:101BB00018962C93AB81BC811496ED91FC911597EE
:101BC000E00FF11FF89E9001F99E300D1124E20FF5
:101BD000F31F8381877F83831496ED91FC91E00F3F
:101BE000F11FE20FF31F86818783C4CFF89ED001D7
:101BF000F99EB00D1124F901EA0FFB1F238121FF8B
:101C0000C4CF23FB222420F823FFBFCF45814F5FA1
:101C10004583EB81FC8124813581F901E00FF11FBF
:101C20005D01AE0EBF1ED50114962C916B817C8197
:101C3000AAE2A29F600D711D11249B01DB011F967A
:101C40005C915417D8F0FC9CC001FD9C900D1124B0
:101C5000E80FF91F8081280F311DF9018785D50113
:101C600017968C93AB81BC811496ED91FC91E00F9B
:101C7000F11F808181608083B22C87CF21813FEF6B
:101C8000320F3183222329F0EB81FC812085215002
:101C90002087EB81FC81A481B581A00FB11FF89E44
:101CA000F001F99EF00D1124AE0FBF1F13962C9179
:101CB0001397277F13962C93AB81BC8114962D919B
:101CC0003C91D901A00FB11FEA0FFB1F238122FF16
:101CD0004FC012962C91129731E0320F12963C931E
:101CE000211105C0EB81FC8121852F5F2187AB810C
:101CF000BC811496ED91FC91E00FF11FF89E50010C
:101D0000F99EB00C1124EA0DFB1D83818061838351
:101D10000E945A22EB81FC8124813581200F311FE2
:101D200049018A0C9B1CA30192010E94C822625E99
:101D30007F4F8F4F9F4FD40114966C93AB81BC8122
:101D40001496ED91FC911597E00FF11FFC9CC001DA
:101D5000FD9C900D1124E80FF91F108214968D91AF
:101D60009C91800F911FA80EB91EF50137827ACF82
:101D70008681878377CFEB81FC818185882309F475
:101D800022C11982E12C85E0F82E9AE5492E512CCA
:101D9000612C712C24E1A22E33243394AB81BC81BD
:101DA00013968C91E81608F00CC1B2E1EB9E80010D
:101DB0001124AB81BC811496ED91FC91E00FF11FD1
:101DC0008281882309F44FC030E020E0EB81FC8160
:101DD00084819581800F911FF29EA001F39E500D8A
:101DE0001124FC01E40FF51FA381B9016F5F7F4F40
:101DF0004B01A0FF61C0A4FB662760F9A4FF5CC093
:101E0000858181508583AB81BC811496ED91FC91D5
:101E1000E00FF11F882349F1DF01A40FB51FF89CE3
:101E2000C001F99C900D1124E80FF91FE081F0E04A
:101E3000E05BFE4F808114969C911497899F802DC2
:101E4000112417968C93AB81BC811496ED91FC9173
:101E5000E00FF11F808181608083698394012330CA
:101E6000310509F0B3CFE39499CF82819FEF980FAA
:101E70009283882329F0EB81FC81818581508187C1
:101E8000AB81BC811496ED91FC911597E00FF11F89
:101E9000F29EC001F39E900D1124E80FF91F2381DB
:101EA0002F7E23831496ED91FC91E00FF11FE80F34
:101EB000F91F86818783C7CFF29E6001F39ED00C05
:101EC0001124FC01EC0DFD1D838181FFC7CF84FB34
:101ED000222420F884FFC2CF85818F5F8583AB8168
:101EE000BC811496ED91FC91E00FF11FEC0DFD1DEE
:101EF00094818913B3CF8781843181F50E945A225E
:101F0000AB81BC811496ED91FC911597E00FF11F08
:101F1000EC0DFD1D34821496ED91FC911597E00FA8
:101F2000F11FF89CC001F99C900D1124E80FF91FD6
:101F300010821496ED91FC91E00FF11FEC0DFD1D48
:101F400086818783AB81BC811496ED91FC91E00F73
:101F5000F11F808181608083298280CF0E945A2274
:101F6000EB81FC8124813581200F311FA9014C0DAB
:101F70005D1D5A834983A30192010E94C822625EBB
:101F80007F4F8F4F9F4FA981BA8114966C93AB817D
:101F9000BC811496ED91FC911597E00FF11FF89C10
:101FA000C001F99C900D1124E80FF91F10821496BE
:101FB0008D919C91800F911FC80ED91EF601A782AA
:101FC000C1CFB981BB2ABB2001F1AB81BC81ED91AE
:101FD000FC9111970680F781E02DCD010F900F90B5
:101FE0000F900F90DF91CF911F910F91FF90EF9085
:101FF000DF90CF90BF90AF909F908F907F906F9029
:102000005F904F903F902F9009940F900F900F90FA
:102010000F90DF91CF911F910F91FF90EF90DF9084
:10202000CF90BF90AF909F908F907F906F905F9078
:102030004F903F902F9008954F925F926F927F92B2
:102040009F92AF92BF92CF92DF92EF92FF920F9347
:102050001F93CF93DF93EC018BEA689F812D1124AE
:10206000869592E1899F70011124EC81FD81EE0D2E
:10207000FF1D982F990F890F681B062F10E044232E
:1020800009F4B5C08FEF820F8F3108F05EC0822F48
:10209000880F880F880F95E0909FD001919FB00D19
:1020A0001124EA0FFB1F8683EC81FD81EE0DFF1DDD
:1020B000AE0FBF1F13968C91139780FF48C081818C
:1020C00091E0980F9183811103C088858F5F888785
:1020D000EC81FD81EE0DFF1D35E0309FC001319F89
:1020E000900D1124E80FF91F8381886083832111EB
:1020F00001C020E2EC81FD81EE0DFF1D85E0809F97
:10210000A001819F500D1124E40FF51F2483EC8161
:10211000FD81EE0EFF1E0F5F1F4F809FF001819F1C
:10212000F00D1124EE0DFF1D1082DF91CF911F9154
:102130000F91FF90EF90DF90CF90BF90AF909F9066
:102140007F906F905F904F9008958FEFA4CF81FFA5
:1021500042C0818191E0980F9183811103C08885ED
:102160008F5F8887EC81FD81EE0DFF1D85E0982E45
:10217000909E5001919EB00C1124EA0DFB1D8381AD
:10218000886083830E945A22CC80DD80CE0CDF1CC5
:10219000CA0CDB1C22E0422E512C612C712CA301B5
:1021A00092010E94C822F60164830E945A220C8088
:1021B000DD81C02DEC0EFD1E0F5F1F4F909EE001D4
:1021C000919ED00D1124CE0DDF1DA30192010E941E
:1021D000C8226883AACF16968C91169717968C936F
:1021E000EC81FD81EE0DFF1D8081816061C085E085
:1021F000809FD001819FB00D1124AE0FBF1F139699
:102200008C9183FF18C081819FEF980F9183882361
:1022100019F0888581508887EC81FD81EE0DFF1DC6
:1022200025E0209FC001219F900D1124E80FF91F88
:102230008381877F8383EC81FD81EE0DFF1D85E027
:10224000809FD001819FB00D1124AE0FBF1F139648
:102250008C9180FF2FC0828191E0980F9283811131
:1022600003C089858F5F8987EC81FD81EE0DFF1D9D
:1022700085E0809F9001819F300D1124E20FF31FB4
:10228000938190619383EC81FD81EE0DFF1DE20F40
:10229000F31F1682EC81FD81EE0EFF1E0F5F1F4FB4
:1022A000809FF001819FF00D1124EE0DFF1D87E04E
:1022B00080833BCF84FF18C082819FEF980F928369
:1022C000882319F0898581508987EC81FD81EE0D85
:1022D000FF1D25E0209FC001219F900D1124E80FD4
:1022E000F91F83818F7E8383AC81BD81AE0DBF1DBD
:1022F00025E0209FC001219F900D1124A80FB91F38
:1023000016961C92EC81FD81EE0DFF1DE80FF91F62
:10231000178266CF0E948A240C94240ACF93DF93FD
:1023200020910802309109022F3F320721F0C901A4
:10233000DF91CF91089580910B0287FF2BC086FF1C
:102340000FC089E090E00E948C11C82F81E090E0DE
:102350000E948C119C2F909309028093080215C053
:1023600089E090E00E948C11C82F81E090E00E94EB
:102370008C1190E4C99F90011124207C31708F73DF
:10238000282B309309022093080280910802909133
:102390000902CECF85FF0CC081E190E00E948C1134
:1023A000C82F82E190E00E948C11C05CDD0BD2CF7F
:1023B00081E090E00E948C1190E0CDCFCF92DF922F
:1023C000EF92FF920F931F93CF93DF93EB017B016B
:1023D00020E2E20EF11C8B016C01C61AD70AC6017D
:1023E000800F911F0E94B222F80181938F01EE1598
:1023F000FF05A9F7CE01DF91CF911F910F91FF90BB
:10240000EF90DF90CF900895CF92DF92EF92FF92FE
:102410000F931F93CF93DF93EB017B0125E0E20E37
:10242000F11C8B016C01C61AD70AC601800F911FDF
:102430000E94B222F80181938F01EE15FF05A9F7E2
:10244000CE01DF91CF911F910F91FF90EF90DF9020
:10245000CF900895CF92DF92EF92FF920F931F9348
:10246000CF93DF93EB017B0126E0E20EF11C8B01A1
:102470006C01C61AD70AC601800F911F0E94B222B2
:10248000F80181938F01EE15FF05A9F7CE01DF91C9
:10249000CF911F910F91FF90EF90DF90CF90089513
:1024A000CF92DF92EF92FF920F931F93CF93DF9320
:1024B000EB017B0128E2E20EF11C8B016C01C61AD4
:1024C000D70AC601800F911F0E94B222F8018193A2
:1024D0008F01EE15FF05A9F7CE01DF91CF911F9176
:1024E0000F91FF90EF90DF90CF9008952F923F9241
:1024F0004F925F926F927F928F929F92AF92BF9214
:10250000CF92DF92EF92FF920F931F93CF93DF93BF
:10251000CDB7DEB7E2970FB6F894DEBF0FBECDBFE2
:102520005C01762E8A01BE016F5F7F4FDC011D9634
:102530008D919C910E945012872D8F7E09F431C19C
:10254000B0E27B1258C1912C812CD5011D968D9142
:102550009C918896BE016F5F7F4F880D991D0E94E8
:102560002A128981682F6F7109F498C1E0901C02CA
:10257000F0901D0286FB332430F8DD24D394B82F6D
:10258000B0724B2E85FDD12C85E0FE013296DE0126
:10259000999601900D928A95E1F75A80F701818111
:1025A000681708F060E0C7010E94B80C682ED701D8
:1025B0001B968C911B972C9110E000E0821778F508
:1025C00091E0980F1B969C931B9718960D911C9168
:1025D000BDE08B9F000D111D1124F80111821082A6
:1025E000D7011D964D915C911E97538342831D9692
:1025F0004D915C911E97558344831D964D915C913E
:102600001E97578346831D964D915C915187408755
:102610001286138694859C7F9B7F9487282EF801D1
:102620008485D0FA81F9848744E0438782E04110B1
:1026300080E0D8011A968C93F7018485982F9170C9
:1026400080FD932DD8011C968C911C9790FB82F9EC
:102650001C968C93652D6F7109F466C0F701828515
:10266000D12CC12C8217A0F491E0980F9287C680DC
:10267000D780F3E08F9FC00CD11C1124D7011F9687
:102680002D913D914C91F60120833183428388AB9B
:10269000D60112968C91129730FA82F912968C9389
:1026A0001297F801848557FA80F98487411009C090
:1026B00012968C91129756FA80F955FA81F9129672
:1026C0008C93D70111968C91681708F060E0C701D0
:1026D0000E94B80CF70124813581E82FF0E0EE0F5D
:1026E000FF1FE20FF31FA081B181F801B183A08326
:1026F000862D90E0880F991F280F391FF9018081DE
:102700009181F6019183808312968D919C9113970C
:102710001496EC91149721E02E0F14962C93E80F49
:10272000F92FF11D48A94083D8011B96DC90E09158
:102730001802F0911902FAABE9AB2E01FAE24F0E42
:10274000511CF80170E0D71609F48EC0D2016D91CA
:102750002D01062F0F7111F1A9A9BAA91A96CC90D3
:1027600090E080E0182F8C1508F07CC09C01220FAF
:10277000331FA9A9BAA91B964D915C91240F351F4F
:10278000D9012D913C91D90114962C9101960213F7
:10279000E9CF128362956695677063837F5F329697
:1027A000D2CFBE016F5F7F4FF501858596850E9470
:1027B0005012D8012D913C91EDB7FEB7B8970FB6E6
:1027C000F894FEBF0FBEEDBFADB7BEB7119688E25D
:1027D000FE01319601900D928A95E1F7D901ED91B4
:1027E000FC91C80109950FB6F894DEBF0FBECDBFAE
:1027F000772009F4A8CEF0E47F125DC0D5011D96C4
:102800008D919C91BE016F5F7F4F80599F4F0E94B9
:102810000412A0910E02B0910F029E012F5F3F4F54
:1028200090E080E050E24C914817190609F00CF452
:1028300040C0F90141919F011196ED91FC911297D1
:10284000E80FF91F46954695469540831196ED9100
:10285000FC911297E80FF91F4081411101C050838C
:102860000196E1CF10E095CF862D90E0880F991F5B
:10287000F70124813581820F931FFC01A081B18172
:102880008D919C9111971596EC91159721E02E0F43
:1028900015962C93E80FF92FF11D2082F6E08F0E8C
:1028A000911C48E48416910409F04FCE7110A3CF17
:1028B000A5CF772019F0B0E57B1245C0D5011D9654
:1028C0008D919C91BE016F5F7F4F8B589F4F0E94EF
:1028D000DE11E0901802F090190210E0F7018285F5
:1028E000181788F5212F30E0C901880F991F03843C
:1028F000F485E02DE80FF91FA081B181E091180265
:10290000F091190211968C91119781708EA71FA6D4
:102910008EA59FA5880F991FE80FF91F81819281CD
:1029200041E050E04C0F5D1F240F351FFC0140813A
:102930005181FA01C280D380F90140816C91F60186
:1029400009951F5FCBCFE2960FB6F894DEBF0FBE9E
:10295000CDBFDF91CF911F910F91FF90EF90DF904E
:10296000CF90BF90AF909F908F907F906F905F902F
:102970004F903F902F900895CF92DF92EF92FF9269
:102980000F931F93CF93DF938C01C62FC07FC0346A
:10299000D9F480911C0290911D020E94E307A0913E
:1029A0000E02B0910F0290E080E02C9128171906DA
:1029B00009F00CF475C01196ED91FC911297E80F97
:1029C000F91F10820196F1CF607D09F442C0C03535
:1029D00009F06AC0C0901802D0901902D0E0D60168
:1029E0001A968C911A97D81708F05EC08D2F90E038
:1029F000880F991F1B96ED91FC91E80FF91FA0819C
:102A0000B18111968C91119713961C9213978B7F1D
:102A10008D7F11968C93119712961C921297E091CC
:102A20001802F091190280FBEE24E0F8F12CC701A6
:102A3000880F991FE80FF91F81819281FC01208185
:102A40003181F901208531856C91F9010995DF5FAC
:102A5000C6CFE0911C02F0911D02238130E090E08E
:102A600080E04FEF82179307A4F4BC01660F771F35
:102A7000A481B581A60FB71F0D90BC91A02D17960C
:102A80004C93179714961C92149715961C920196C6
:102A9000E9CF138212861386CC2309F480CF97CF17
:102AA000CC2309F497CF93CFA801445F5F4F6C2FDD
:102AB0008091100290911102DF91CF911F910F919F
:102AC000FF90EF90DF90CF900C947612CF93DF932E
:102AD000EC018C899D898617970749F07D8B6C8B5B
:102AE0008D859E85860F971F0E94B2228E8B8E89C0
:102AF000DF91CF9108958331910588F4813191055B
:102B000030F48130910519F08930910531F42FEFBF
:102B10003FEF30930902209308020C94150A8D317F
:102B20009105D9F7677F60930B022091F2012F7313
:102B3000362F307C232B2093F201E9CFBF92CF9226
:102B4000DF92EF92FF920F931F93CF93DF938B014E
:102B5000B42E690182FF23C083FF17C061E0C80162
:102B60000E94420A8823D9F16B2DC8010E947B156F
:102B70008B1135C0F601DF91CF911F910F91FF901E
:102B8000EF90DF90CF90BF90099460E0C8010E9461
:102B9000420A882321F1C8010E948C11E9CF842FB9
:102BA0008770C1E0D0E07E0101C0EE0C8A95EAF7A3
:102BB000D42FD870CB010E948C11C82FB4FE1CC03A
:102BC00061E0C8010E94420A882349F0DD2389F0B0
:102BD000CE296C2FC8010E947B158C1759F2DF910A
:102BE000CF911F910F91FF90EF90DF90CF90BF900A
:102BF0000895E094CE21EDCF60E0C8010E94420A22
:102C0000882369F3CE21DD2319F0C111B3CFE7CFBB
:102C1000CC2309F4AFCFE3CFCF92DF92EF92FF92B4
:102C20000F931F93CF93DF937C016B01C42F122F5F
:102C3000D42FD07E8091F20187FF2CC0D03EC1F509
:102C40008091F3018823A1F190E00E948C11D82F8C
:102C50008091F30190E001960E948C11982F8D2FA6
:102C6000E816F90629F56C2F70E0762F662766279F
:102C70007370612B6F5F7F4F24E43AE0402F8C2FFD
:102C8000DF91CF911F910F91FF90EF90DF90CF9048
:102C90000C949E1580FD32C0D03609F464C088F4CF
:102CA000D03209F447C0D03409F45DC0DD2379F196
:102CB000DF91CF911F910F91FF90EF90DF90CF9018
:102CC0000895D03A09F483C090F42C2F2F7141E07D
:102CD00050E0D03869F7B601C701DF91CF911F915D
:102CE0000F91FF90EF90DF90CF900C94080AD03CAA
:102CF00009F476C0D03E09F4B6CFDACF0E948E1127
:102D00008E159F0549F2E114F10431F2D1CF8C2FD9
:102D10008E7071F680E090E0892B51F28C2F8170DB
:102D2000DF91CF911F910F91FF90EF90DF90CF90A7
:102D30000C940000CF71CF3109F0BACF412F4F77FB
:102D400071F0413071F0111F1127111F212F30E058
:102D50000FE710E0B601C7010E94F209A9CF41E0D8
:102D6000F2CF40E0F0CF2C2F30E08C2F8F718130EC
:102D700029F030F0803121F08131F9F440E001C0D8
:102D800041E025FB222720F90DE110E030E0B601FB
:102D9000C7010E94F20980E090E0892B09F488CFF6
:102DA0004C2FB601C701DF91CF911F910F91FF907A
:102DB000EF90DF90CF900C940000C901880F991F0D
:102DC0008E71C4FB442740F9482B4250DACF2C2F98
:102DD0002F7043E050E0C4FF7ECF42E050E07BCF55
:102DE000CF71CE3139F0CF3109F062CF212F45E0DC
:102DF00050E071CF212F44E050E06DCFFF920F9350
:102E00001F93CF93DF93EC01F62E08811981C8013F
:102E10000E94B222F81621F06F2DC8010E94BA223A
:102E2000CE01DF91CF911F910F91FF9008952F92C6
:102E30003F924F925F926F927F928F929F92AF924A
:102E4000BF92CF92DF92EF92FF920F931F93CF9397
:102E5000DF93CDB7DEB7E4970FB6F894DEBF0FBEB1
:102E6000CDBF7C01462E542E8E010F5F1F4FB8013F
:102E7000DC011D968D919C910E9450126E01B9E269
:102E8000CB0ED11C460196EFA92E93E0B92E360148
:102E9000C5010E94B222F40181934F01FFEFAF1AE6
:102EA000BF0AA11484E0B80699F7511001C059A4D3
:102EB000D7011D96AD90BC901E978A8118166CF5AF
:102EC00089858D3051F58885803139F5411025C0CF
:102ED000B501695F7F4FED91FC910084F185E02D94
:102EE00020E040E1C7010995E4960FB6F894DEBFF3
:102EF0000FBECDBFDF91CF911F910F91FF90EF904B
:102F0000DF90CF90BF90AF909F908F907F906F9009
:102F10005F904F903F902F900895A114B4E0BB06AE
:102F200040F460E0C5010E94BA22EFEFAE1ABE0A7B
:102F3000F4CF89A5851159A686EFA82E83E0B82E77
:102F4000BCAAABAAD6016D916D01CE01C3960E94B9
:102F5000FE16BFEFAB1ABB0AA114E4E0BE0681F770
:102F600088E2D8011D928A95E9F78DE0898780E192
:102F7000888782E08E8FF7018789908DDC01ED9143
:102F8000FC910190F081E02D652D0995009729F0C5
:102F90008038910508F08DC08A83F7018789908D6C
:102FA000DC01ED91FC910280F381E02D652D099506
:102FB000009729F08038910508F084C088A3F701B4
:102FC000C584D6845801C01AD10AC6018A0D9B1D3A
:102FD0009CAB8BABD5016D915D01CE01C3960E9478
:102FE000FE166A147B0489F7B12CA12C412CF70141
:102FF00032963F011801F6E02F0E311CD7011D96C5
:103000008D919C918896B8018A0D9B1D0E942A1271
:1030100086E0F301D80101900D928A95E1F75520E1
:1030200079F0F7018789908D009751F0DC01ED91DF
:10303000FC910480F581E02D9801442D652D0995C2
:10304000F701C584D684F8E2CF0ED11CCA0CDB1C74
:103050004801C01AD10AC601880D991D9CAB8BABE3
:10306000D4016D914D01CE01C3960E94FE16281425
:10307000390489F74394B6E0AB0EB11CECE04E1274
:10308000BDCFD7011D968D919C91B80180599F4F5E
:103090000E940412F701828590E0F8019F01201B35
:1030A000310B28173907ACF4D70119962C912193CD
:1030B000F5CF2E8D22622E8F23E02A8390549A8B97
:1030C0008B8B6BCF2F8D21602F8F905499A38AA368
:1030D00076CF5520F1F0F7018789908D892BC9F0C3
:1030E000D12CD7011A968C911A97D81690F457962E
:1030F0008D919C91DC01ED91FC910680F781E02D92
:103100004D2D652D0995F801ED0DF11D8083D394AA
:10311000E8CFF701C584D6844601F0E78F0E911CF5
:1031200085E7C80ED11C58019CAA8BAAD5016D91C8
:103130005D01CE01C3960E94FE16BFEF8B1A9B0A5B
:10314000C814D90489F7F70185859685B8018B588D
:103150009F4F0E94DE11D7011B962C91C8018096CB
:103160006801F60121936F018E179F07D1F7552053
:10317000E1F0D70157968D919C91892BB1F0B12C3C
:10318000F7018485B81688F48789908DDC01ED916C
:10319000FC910084F185E02D4B2D652D0995F801FA
:1031A000EB0DF11D8083B394EBCFF701E584F6843A
:1031B000E01AF10AC7018B589F4F7C01C701800FAD
:1031C000911F9CAB8BABD8016D918D01CE01C39645
:1031D0000E94FE16C016D10689F786CEAF92BF9226
:1031E000CF92DF92EF92FF920F931F93CF93DF93D3
:1031F0001F92CDB7DEB77C01C42E00911002109152
:103200001102D801ED91FC910190F081E02D21E0B7
:10321000AE014F5F5F4FC80109955C010196A1F4B3
:10322000D12CF701828181113EC089818F70863057
:10323000A8F5833010F48130B1F5DD20A1F1C7018C
:103240000E944E0A698148C0D801ED91FC9102802C
:10325000F381E02D2C2D4981B701665F7F4FC801B6
:103260000995D82E8823E1F2D801ED91FC910680D2
:10327000F781E02D4981B501C8010995C81661F0B3
:10328000D801ED91FC910084F185E02D29814C2D30
:10329000B501C8010995C5CF1982C3CF873081F028
:1032A00010F08B3050F28D2D0F90DF91CF911F9148
:1032B0000F91FF90EF90DF90CF90BF90AF90089567
:1032C000C7010E944E0A40E061E080911002909197
:1032D00011020E94171760E0C7010E94BC14E3CFDF
:1032E000CF93DF9300D0CDB7DEB7FB012F7027302F
:1032F000B9F0DC0154962D913C91559762177307F4
:1033000011F456964C93642FDC011D968D919C917F
:10331000E80FF91FFA83E983CE0101960E94FE1699
:103320000F900F90DF91CF910895BF92CF92DF92CF
:10333000EF92FF920F931F93CF93DF937C018091C5
:10334000F4018823B1F00E9496030091F5011091D9
:10335000F6012091F7013091F801601B710B820B8F
:10336000930B653171058105910518F080E00E948D
:103370002F0D8091DE018823B1F1F89488E0EAEE08
:10338000F1E0AEE1B2E001900D928A95E1F7109282
:10339000DE01789480911E02E82FF0E0E05EFD4FA0
:1033A000863018F411928F5FFBCF80E090E0892B7C
:1033B00021F08EE192E00E940000809120028111B4
:1033C0004AC090912102911146C080E090E0892B83
:1033D00019F080E00E9400008091F4018823B9F187
:1033E00081E00E94C109D70119968C91882371F060
:1033F000C70104960E946E0A811108C060E0F701BF
:1034000083810E94CA00D70119961C92009118026C
:1034100010911902C80105960E946E0A811134C2EA
:10342000C0E0F8018081C81708F021C2EC2FF0E05D
:10343000EE0FFF1FE00FF11F81819281DC01ED9102
:10344000FC910284F385E02D0995CF5FEACF81E0FE
:103450000E942F0DC8CF9091F401992309F482C0E6
:103460008057803108F07BC081E00E94C109C09183
:103470001E028091FB01C8130AC04C2F50E06DEF73
:1034800071E080E292E00E948F24892B61F010921B
:10349000FA0188E0EEE1F2E0ABEFB1E001900D92CD
:1034A0008A95E1F7A0CF8091FA018F5F8093FA01AE
:1034B000C330E9F520912002822F877010912102FC
:1034C000853029F41093F9010E94660A8CCFCDE172
:1034D000D0E0843089F0C82FD0E0843060F480914F
:1034E000F901882341F08150990B880F991F880FAB
:1034F000991FC80FD91F219623FF0EC061E0CE018E
:103500000E94420A882309F46ECF612FCE010E94E7
:103510007B15181368CFD8CF60E0CE010E94420A15
:10352000882309F460CFCE010E948C11F2CFC43001
:1035300009F059CF80912002682F70E0762F66271E
:103540006627737090912102692B6F5F7F4F2CE685
:103550003AE0409122028C700E949E1544CF80E098
:103560000E942F0DE0912002EF3F61F48091210233
:10357000811139CF80E090E0892B09F434CF0E948B
:10358000000031CFE7FD0DC00091230220912202FF
:103590004091210270E060E08E2F90E00E940C16B6
:1035A00022CFE03C08F052C19091F20197FF1BCF6F
:1035B00080912102682F70E0EB01C095D095CC0F6F
:1035C000DD1FCC0FDD1FC07CD170EF73CE2B759546
:1035D0006795262F2370B22E20911E02253039F5D3
:1035E0008C788C3021F50E948E118C179D0721F06C
:1035F000CF3FD14009F0F7CE8091210290E0982F83
:10360000882788279370C0912202C80FD92FD11D17
:1036100021961091230261E0CE010E94420A612F9F
:10362000882309F4E0CECE010E947B15DCCE6E012A
:10363000A1E0CA1AD108CC0CDD1CCC0CDD1CCB28B7
:1036400086010F5F1F4F80910A028823F9F096FFD1
:1036500041C0C80160E071E00E944B23682F81E007
:1036600090E00E947B15C80117FF02C081509F4F58
:10367000692F89E090E00E947B1580E090E0892B23
:1036800019F0C8010E94000010920A028091F20114
:1036900080FD39C080911E02843009F04EC08091B7
:1036A00021028978813009F09ECE80E090E0892B5C
:1036B00029F060912202C8010E94000080E090E0A1
:1036C000892B09F490CE409122026B2DC8010E94F3
:1036D000000089CEBE016F73772781E090E00E94E1
:1036E0007B15BE0146E0759567954A95E1F789E03F
:1036F00090E00E947B1580E090E0892B29F2CE01BA
:103700000E940000C1CF86FF0CC00E948E1180175E
:10371000910709F4BFCF0D3FB7E01B070CF0BACFFC
:1037200062CE0E948E118C179D0709F4B3CFCF3F54
:10373000E1E0DE0709F4AECF56CE833069F5409163
:103740002102F42FF170CF2E43FBDD24D0F880E06E
:1037500090E0892B31F047702D2DBE01C8010E94E9
:1037600000008091F20186FF0BC080E090E0892B81
:1037700009F439CE4D2D6C2DC8010E94000033CEC6
:1037800080E090E0892B09F42ECE2D2D4C2D6B2D51
:10379000CE010E94000027CE863009F024CE809111
:1037A0002102982F9978913021F08F78803809F094
:1037B0001ACE8091F20186FF25C00E948E118017DB
:1037C0009107E1F48091220290E0382F22272227EE
:1037D0003370C0912302C20FD32FD11D21961091B7
:1037E00024029595879595958795837099278230C2
:1037F000910589F0039709F40ECFF5CD0D3F1740E1
:103800000CF7F1CD0E948E118C179D07D9F2CF3F96
:10381000D140C1F2E8CD14FFE6CD61E0CE010E94B7
:10382000420A882309F4DFCDCE010E948C11912F2A
:10383000977061E070E001C0660F9A95EAF713FF98
:1038400002C0682BF0CE60956823EDCEE83E08F00C
:10385000CACDE05CFF0B80912102009124022091EF
:1038600023024091220261E070E09E2F97CE0E94D9
:103870009603685D7F4F8F4F9F4FF8016683778374
:103880008087918783E08583DF91CF911F910F918E
:10389000FF90EF90DF90CF90BF9008951F920F920E
:1038A0000FB60F9211242F933F938F939F93AF9353
:1038B000BF938091CE019091CF01A091D001B091A2
:1038C000D1013091CD0123E0230F2D3758F501961A
:1038D000A11DB11D2093CD018093CE019093CF0106
:1038E000A093D001B093D1018091D2019091D301E6
:1038F000A091D401B091D5010196A11DB11D809375
:10390000D2019093D301A093D401B093D501BF917C
:10391000AF919F918F913F912F910F900FBE0F907C
:103920001F90189526E8230F0296A11DB11DD2CF36
:103930001F920F920FB60F9211242F933F934F9324
:103940005F936F937F938F939F93AF93BF93EF9307
:10395000FF93E0910201F09103010995FF91EF912E
:10396000BF91AF919F918F917F916F915F914F9197
:103970003F912F910F900FBE0F901F9018951F929F
:103980000F920FB60F9211242F933F934F935F9393
:103990006F937F938F939F93AF93BF93EF93FF9317
:1039A000E0910001F09101010995FF91EF91BF9124
:1039B000AF919F918F917F916F915F914F913F91C7
:1039C0002F910F900FBE0F901F901895CF93DF93FC
:1039D000CDB7DEB7FC018AA185FF14C02E89205C1B
:1039E000330B8F89922F978786878BA180FF0DC01D
:1039F0002DA1205C330B8EA1922F918B808BDF91B8
:103A0000CF9108958E8190E0EECF8CA190E0F5CF1C
:103A1000CF93DF93CDB7DEB728E2FE013596DF0105
:103A200001900D922A95E1F70C97DF91CF910C94BC
:103A3000E61C6F70693011F481E0089580E008950C
:103A40000A970C94191DE62FEF70E150EA3018F533
:103A5000F0E0E35DF24E0C945F23371D4B1D391DE2
:103A6000391D4D1D4B1D4B1D371D371D6A1D81E036
:103A70000895E0911C02F0911D029181842F8F71B5
:103A8000981748F0407EE0910E02F0910F0281E01D
:103A90009081941710F580E020C0242F207E30E024
:103AA00085E0359527958A95E1F74F71E0911802E9
:103AB000F091190281E09285941708F480E0E0917A
:103AC0000E02F0910F0291E03081321708F490E07D
:103AD0008923089581E04230F0F608950A970C9406
:103AE000231D0895CF93DF9300D000D000D01F9204
:103AF000CDB7DEB7789484B5826084BD84B581602B
:103B000084BD85B5826085BD85B5816085BD8091A8
:103B10006E00816080936E00109281008091810020
:103B20008260809381008091810081608093810018
:103B3000809180008160809380008091B1008460DA
:103B40008093B1008091B00081608093B00080913B
:103B50007A00846080937A0080917A0082608093FA
:103B60007A0080917A00816080937A0080917A0057
:103B7000806880937A001092C10080E480937C007A
:103B800080917A00806480937A0080917A0086FD2B
:103B9000FCCF8091780060917900762F682F072EF6
:103BA000000C880B990B611571058105910511F0C9
:103BB0000E94A92282E090E00E9465233C0181ECF2
:103BC00091E0D3018D939C93709215026092140240
:103BD00082E090E00E9465239A83898383EB91E0E1
:103BE000E981FA8191838083F0931302E0931202BA
:103BF00086E190E00E9465237C0186E1D7011D9259
:103C00008A95E9F7F70114828DE891E0918380832A
:103C100085EA91E0938782878DEA91E09587848792
:103C2000F0921702E09216028DE090E00E94652368
:103C30006C01DC0115961C92909319028093180276
:103C4000C3010E94B60CF601828790E0880F991F8D
:103C50000E946523D6011C969C938E931B971B8212
:103C60001C82B12CF6018285FB81F817F0F4D30198
:103C7000ED91FC910480F581E02D6B81C3010995E4
:103C8000892B29F4B394EB81EF5FEB83EBCFD30166
:103C9000ED91FC910280F381E02D6B81C3010995C8
:103CA000BC81B81780F78C83EECFFC81FF73AF2EF9
:103CB00081E0D6018C938EE090E00E9465239D8385
:103CC0008C838BE791E0EC81FD819183808386E09A
:103CD0008F01085F1F4FD801E82F1D92EA95E9F781
:103CE0009FEFAC81BD8119969C9319971296BC9257
:103CF000129715969C9115979E7F15969C93B89E4A
:103D0000C00111240E946523EC81FD81838394838B
:103D10009C0190E0502F412FB91661F086E0E52F0D
:103D2000F42FD90101900D928A95E1F79F5F2A5FE8
:103D30003F4FF2CFAC81BD8116961C921697179615
:103D40001C921797F601B283A183AA2009F479C1C6
:103D50008A2D90E0029663E070E00E944B23862E4D
:103D6000572E962E82E080838DE890E00E94652396
:103D70008C0189E691E0D80111969C938E93F8010D
:103D80003A96FD83EC8385E011928A95E9F786E007
:103D900012968C93129713968C92A82CB52C82E1D4
:103DA000B82FBA9DC001BB9D900D11240E946523C0
:103DB000F801958384831086118690E080E040E0CE
:103DC00055E02C812B833D813C83D8011496ED91E5
:103DD000FC911597E80FF91F20812160208314962C
:103DE000ED91FC911597E80FF91F11821496ED9152
:103DF000FC91E80FF91F128230E020E0F801A48165
:103E0000B581A80FB91F529FB001539F700D1124A7
:103E1000A60FB71F1396EB81FC81652F01900D92C1
:103E20006A95E1F72F5F3F4F2330310539F74F5F38
:103E30004296491550F286E190E00E9465239D83E9
:103E40008C83DC0111961C92119718961C92FC0130
:103E50001786108A118A128A1686138681E0848753
:103E600092E0958780834501880C991C8A0C9B1CE5
:103E700095828482C4010E946523AC81BD811A961B
:103E80009C938E931997009709F425C1A40170E0C3
:103E900060E00E949C24EC81FD81B382A28286E0D6
:103EA00090E0EC81FD81978386838181882341F0B6
:103EB00061E086E00E94160160E086E00E94CA0090
:103EC000E1E0F1E0E491F0E0EE0FFF1FEF50FF4F73
:103ED00085919491AC81BD8154969C938E93539718
:103EE000E3EEF0E0E4915596EC935597F801B78333
:103EF000A68316968D919C9197FD0AC061E00E9461
:103F0000160160E0AC81BD8116968C910E94CA00BA
:103F100081E0EC81FD818183312C212C512C412CBD
:103F20000E945A2224E030E040E050E00E94C82283
:103F30004B015C01F4E08F0E911CA11CB11C8B8223
:103F400024E130E0E1E0F0E041E0C801820D931DA2
:103F50009D838C83AC81BD81AE0FBF1FBF83AE83B9
:103F6000C901B4010E944B23AE81BF811F966C939F
:103F700081E0840F31962C5E3F4FBB81B81708F06B
:103F8000B5C052E0B52EB40E0E945A2222E030E0B5
:103F900040E050E00E94C82272E0972E960EA12CBD
:103FA0002AE2249DF001259DF00D1124E00FF11F60
:103FB000FD83EC830E945A2222E030E040E050E092
:103FC0000E94C8226E5F2B2D30E0EC81FD81E20F54
:103FD000F31F178682E090E0220D331DF901E80FF0
:103FE000F91FE00FF11F44E14687482F01965FEF6C
:103FF000580F651798F7B40E0E945A22EC81FD8184
:10400000EB0DF11D17868FEF808BB394B394A394BF
:10401000A91480F2AC81BD811F96BC92BFEF4B1AF0
:104020005B0AEAE22E0E311CF3E04F16510409F050
:1040300077CFC8010E945404D60114961C930E93A6
:1040400013971B82F6018285FB81F81708F079C06F
:10405000D301ED91FC910280F381E02D6B81C301CE
:1040600009958C83D301ED91FC910480F581E02DBD
:104070006B81C3010995BB80B3940097C9F585E0B6
:1040800090E00E9465238C01FC011382B4822C8194
:10409000208381818C7F8B7F81831282E091180243
:1040A000F091190281819281DC01ED91FC910190E6
:1040B000F081E02D622F0995BB818B2F90E0880F56
:1040C000991FF6010384F485E02DE80FF91F118391
:1040D0000083BB82B7CFAC81BD8115961C921E9226
:1040E000149713961C921E921297D9CE482F32CF56
:1040F000019779F785E090E00E9465238C01DC014F
:1041000013961C9213971496BC921497EC81EC931F
:1041100011968C91119781608D7F8B7F11968C9376
:10412000119712961C92E0911802F0911902838166
:104130009481DC01ED91FC910190F081E02D6C8186
:10414000BACF89E190E00E946523FC019C012E5FBB
:104150003F4F86E0D9011D928A95E9F711861386B3
:104160008BE591E091838083DD24DA94D08A8FEF10
:104170009FEF928B818B138A958B848B168AF09399
:104180001102E09310021686158629813A81308F3C
:10419000278B8CE0808785E08287A0911802B09100
:1041A00019021A968C91848741E060E0CF010E9449
:1041B00017170091100210911102D8011A96CC9095
:1041C00083E090E00E9465239A83898390930F0295
:1041D00080930E02FC01C0828C2D90E00E9465232A
:1041E000A981BA8112969C938E93119787E090E0F3
:1041F0000E946523FC0181E090E09183808393839A
:104200008283148215821682F0931B02E0931A02B5
:10421000F801C08482E190E00E9465239A8389833B
:10422000DC011A961C921A971B961C921B971D96DE
:10423000DC921D971E961C92FC011786108A118A2B
:1042400090931D0280931C02C0828DE181838C2D8E
:10425000880F8283948591609487138290E0880F01
:10426000991F0E946523A981BA8114968C93149793
:1042700015969C93FC0190E080E0A981BA8112968A
:104280002C912817190629F024F011921192019609
:10429000F4CF83E0D82ECD9CC00111240E94652369
:1042A000E981FA8197838683FDE0CF9EC0011124C6
:1042B0000E946523A981BA8119969C938E931897C1
:1042C0001A961C921A971B961C92A701445F5F4F87
:1042D00060E0C8010E947612F894F0920D02E0921C
:1042E0000C0284E0F701838361E00E94160160E024
:1042F000D70113968C910E94CA0021E0F701228316
:104300001092030282E080930402EDEFF0E0E4916A
:10431000F0E0EE0FFF1FED52FF4F859194919093C7
:10432000060280930502EFEDF0E0E491E0930702CE
:1043300060E082E00E941601ECEDF1E086E1DF0131
:104340001D928A95E9F782E990E09093DB018093D2
:10435000DA0182E590E09093D9018093D801109220
:10436000F201B1E0B093F3018FEF9FEF9093090258
:104370008093080210920A02D092D701809107021E
:104380008093D60163E070E0809103020E94A70051
:104390008DE190E00E948C11682F6F738DE190E0A9
:1043A0000E947B1580930B0260E087E090E00E9402
:1043B0007B1560E088E090E00E947B1580E00E9421
:1043C0002F0DF7011282E0911C02F0911D0281E095
:1043D000D70150962D913C91232B09F480E0248540
:1043E000922F917020FD982F848590FB81F984870E
:1043F000CF010E94E30778948091160290911702F2
:10440000DC01ED91FC910484F585E02D0995E0E057
:10441000F0E0EF2B89F30E940000EECF8F929F9285
:10442000AF92BF92CF92DF92EF92FF92CF93DF9342
:10443000EC01688179818A819B8161157105810513
:10444000910521F464E279ED8BE597E02DE133EFFE
:1044500041E050E00E94C82249015A019B01AC0191
:10446000A7EAB1E40E94E7226B017C01ACEEB4EF55
:10447000A50194010E94F522C60ED71EE81EF91E62
:10448000F7FE06C081E0C81AD108E10880E8F80A02
:10449000C882D982EA82FB82C701B6019F77DF9189
:1044A000CF91FF90EF90DF90CF90BF90AF909F9013
:1044B0008F9008958F929F92AF92BF92CF92DF928A
:1044C000EF92FF92609104017091050180910601C5
:1044D00090910701611571058105910521F464E250
:1044E00079ED8BE597E02DE133EF41E050E00E945C
:1044F000C82249015A019B01AC01A7EAB1E40E941C
:10450000E7226B017C01ACEEB4EFA50194010E949F
:10451000F522C60ED71EE81EF91EF7FE06C081E082
:10452000C81AD108E10880E8F80AC0920401D092C4
:104530000501E0920601F0920701C701B6019F77DD
:10454000FF90EF90DF90CF90BF90AF909F908F90B3
:104550000895609304017093050180930601909380
:1045600007010895F999FECF92BD81BDF89A992768
:1045700080B50895262FF999FECF1FBA92BD81BD4F
:1045800020BD0FB6F894FA9AF99A0FBE01960895D5
:10459000052E97FB1EF400940E94DF2257FD07D0E2
:1045A0000E94FA2207FC03D04EF40C94DF225095AF
:1045B0004095309521953F4F4F4F5F4F089590950F
:1045C0008095709561957F4F8F4F9F4F08950E9402
:1045D0001C23A59F900DB49F900DA49F800D911D4D
:1045E00011240895B7FF0C94E7220E94E722821B52
:1045F000930B0895A1E21A2EAA1BBB1BFD010DC04F
:10460000AA1FBB1FEE1FFF1FA217B307E407F50782
:1046100020F0A21BB30BE40BF50B661F771F881F5E
:10462000991F1A9469F760957095809590959B01F4
:10463000AC01BD01CF010895A29FB001B39FC0019D
:10464000A39F700D811D1124911DB29F700D811DBE
:104650001124911D0895991B79E004C0991F9617A4
:1046600008F0961B881F7A95C9F780950895AA1BB4
:10467000BB1B51E107C0AA1FBB1FA617B70710F04D
:10468000A61BB70B881F991F5A95A9F7809590957F
:10469000BC01CD01089597FB072E16F4009407D0B6
:1046A00077FD09D00E94372307FC05D03EF4909592
:1046B00081959F4F0895709561957F4F0895EE0FF6
:1046C000FF1F0590F491E02D09940F931F93CF9352
:1046D000DF938230910510F482E090E0E0912802AF
:1046E000F091290230E020E0B0E0A0E0309799F4AA
:1046F0002115310509F44AC0281B390B2430310536
:10470000D8F58A819B816115710589F1FB0193833D
:104710008283FE0111C040815181028113814817BB
:104720005907E0F04817590799F4109761F012966D
:104730000C93129713961C933296CF01DF91CF9171
:104740001F910F9108950093280210932902F4CF2E
:104750002115310551F04217530738F0A901DB014B
:104760009A01BD01DF01F801C1CFEF01F9CF9093AC
:10477000290280932802CDCFFE01E20FF31F81931F
:1047800091932250310939832883D7CF2091260273
:1047900030912702232B41F420910A0130910B0123
:1047A00030932702209326022091080130910901BD
:1047B0002115310541F42DB73EB740910C015091C0
:1047C0000D01241B350BE0912602F0912702E21720
:1047D000F307A0F42E1B3F0B2817390778F0AC0124
:1047E0004E5F5F4F2417350748F04E0F5F1F509301
:1047F000270240932602819391939FCFF0E0E0E05F
:104800009CCFCF93DF930097E9F0FC01329713829E
:104810001282A0912802B0912902ED0130E020E03F
:104820001097A1F420813181820F931F20912602DD
:10483000309127022817390709F061C0F093270249
:10484000E0932602DF91CF910895EA01CE17DF07AA
:10485000E8F54A815B819E0141155105B1F7E901F7
:10486000FB83EA8349915991C40FD51FEC17FD07CB
:1048700061F4808191810296840F951FE9019983EB
:104880008883828193819B838A83F0E0E0E01296A3
:104890008D919C9113970097B9F52D913C911197AB
:1048A000CD010296820F931F20912602309127029C
:1048B0002817390739F6309751F5109229021092CE
:1048C0002802B0932702A0932602BCCFD383C283D1
:1048D00040815181840F951FC817D90761F44E5F3D
:1048E0005F4F88819981480F591F518340838A8186
:1048F0009B81938382832115310509F0B0CFF0931A
:104900002902E09328029ECFFD01DC01C0CF138273
:104910001282D7CF81E090E0F8940C94A324FB019D
:10492000DC0104C08D910190801921F44150504068
:10493000C8F7881B990B0895DC0101C06D934150A5
:0A4940005040E0F70895F894FFCF0F
:10494A00A203A2030100000000002A0280005D0009
:10495A00242603005D002500000047000600000031
:10496A004B000200000069004708090A69000B0CA5
:10497A0000006A000D0F110078000E000000790097
:10498A00500000005400120000000005090D151D1A
:10499A000001020304050700000000AC0AA20A9500
:1049AA000A6615701900000000E207DC051C1054A5
:1049BA0004A4033E0DA303000000009C07C4071EC5
:1049CA0007E107D8062A06A303000000003A0C0EE6
:1049DA000CEE187F0B550BA3039519231D191DE621
:1049EA001CF6FF00006E1D201DF4FF0000081D00CC
:1049FA00000000A40CA10C630C5D0C570C00000015
:084A0A0000B60CB00CA70C0073
:00000001FF
